:1000000095C1AFC1AEC1BAC3ACC1ABC1AAC1A9C190
:10001000A0C2A7C1A6C1A5C1A4C1A3C1A2C1000419
:10002000FFF112FCFA0FF706F00300FF00FD1000CD
:10003000FCEE0DF9FB04030A020FF92107F612E5A5
:1000400002FD10FBE1FBEF08EAFAF8F509F701F70A
:10005000F6FD061B06FFF3E906F410051809080E65
:10006000F705EC0AE7FBF404F5EF08F70BEE17F7DA
:100070000E00090B0410EA0DF90CF604E6EE03F984
:100080000EEF03FF12FB0B0E0007F108F9FBFBFE5E
:10009000F9EEFDFC04FCFE0B0C040103F8F3FE0278
:1000A00007000B0601FDFF0901FFFAFFFD0BF4FE3F
:1000B000F6FC020404FD0CFA04E90408FC07FAFE4D
:1000C000FFFCF5F6F606FBFB03FF0309FF02000049
:1000D0000CFD04FDFEFA0C00020FFF06F706FCFF04
:1000E000FDF0FFFCFCFEF9F90804010802FB00F832
:1000F00001050600F501F40008FAFDFDF9FF03FB18
:1001000005FC0410F908040107FAF4F9070101FDE0
:1001100000010201F7FB07FDFAFDF904FE080700E4
:100120000B01FBFDF5F705FDFDFCFD05020AFAFDDF
:1001300008F9F8FE03FF05020103020801FDFEF9BC
:10014000FD01FDFF0201FAFC00FB010101010202B9
:10015000F90106FEFD0702FFF7FA03FE01FFFFF9B2
:100160000109FFFD0306FB04FDFF03F3FD0205FB90
:1001700002F80301FC02FA08F70105FBF9FF04FF8E
:10018000FD0400FDFFFF04FFFF03040101F9040665
:10019000FEFCFC0002FEFD03F902FEFFFE0200FB76
:1001A000FAF903FE05FA0402FE07FFFE0100FB0256
:1001B000FD03000204FB010203FD03FDFE03FCFF3F
:1001C000FE01FCFAFF04FDFDFEFB01FD06FE000240
:1001D0000100FE01F705FB0404FE06FF00FC04021B
:1001E000FFFF01FDFEFFF901FFFA01FDFD02FB0328
:1001F000FEFD03FFFE010100000002FE010500FEFE
:1002000003FE00FE00FFF900FFFFFB02000200FEFC
:1002100001FD00FEFCFF0301FFFDFEFFFF01FE01EB
:100220000302020000FE03FBFD02FFFDFD0501FFCE
:10023000FF000100FDFE0001FF0002FEFFFE03FDC6
:10024000FE01FEFFFF0301FEFEFFFFFF00FF0001B6
:1002500000000403FEFFFE000000FEFB00000001A2
:10026000FDFEFFFEFD00FEFE01FE000001FF00019D
:1002700002FEFF0000020101FF02FF00FF01FE007D
:10028000FFFD01FE00FEFF0000FFFF0000FFFF007A
:100290000000000000000001010102020304050546
:1002A0000607090A0B0C0E0F1112141517191B1D46
:1002B0001F212325282A2C2F313436393B3E414338
:1002C00046494C4F5255585A5D6164676A6D707368
:1002D00076797C808386898C8F9295989B9EA2A547
:1002E000A7AAADB0B3B6B9BCBEC1C4C6C9CBCED047
:1002F000D3D5D7DADCDEE0E2E4E6E8EAEBEDEEF0D7
:10030000F1F3F4F5F6F8F9FAFAFBFCFDFDFEFEFE5A
:10031000FFFFFF000000003800000000003700026F
:1003200002020202020102040810200011241FBE72
:10033000CFE5D2E0DEBFCDBF10E0A0E6B0E0E8E759
:10034000F9E002C005900D92A638B107D9F721E077
:10035000A6E8B0E001C01D92A43AB207E1F79DD231
:1003600009C34ECEEF92FF920F931F93CF93DF936B
:1003700080916000813009F459C050F0823009F456
:1003800092C0DF91CF911F910F91FF90EF90089550
:1003900000919300C091A0008091920090E0EE2423
:1003A000EA94F12CD0E09701281B390BC901BE015A
:1003B000D0D2492F90939300292F30E0A0918D0047
:1003C000B0918E008091900090E08D559F4FFC0180
:1003D000808190E0B901BDD2192F8B2F99278D55BF
:1003E0009F4FFC018081B7016C1B7D0B90E0B1D267
:1003F000910F90938C00041730F480E090E4909378
:10040000900080938F00201B310937FF03C0319586
:1004100021953109243008F4B4CF80E0922F8A0F5F
:100420009B1F90938E0080938D00ABCF2091910005
:100430003091920036952795369527958091A000AA
:100440008456990B75E0880F991F7A95E1F7281764
:10045000390720F0109292001092910020919100A3
:1004600030919200F901F695E795F695E795E25EF1
:10047000FF4F649180918B0090E08D559F4FFC0160
:10048000808170E090E065D290938900E0918800CF
:10049000F0E0232F3327ED55FF4FE20FF31F80814C
:1004A00080938C006ECF80918B0090E02091A00013
:1004B0002817190648F42091920030E02D553F4F3F
:1004C000F9012081209389002091900030E02D5582
:1004D0003F4FF90140818D559F4FFC018081480FAE
:1004E0005527551F20918E0030E02D553F4FF901C3
:1004F0008081480F511D2091870030E02D553F4FDE
:10050000F9018081840F952F911D9595879595957B
:100510008795C6CF90E0FC01EB5DFC4F2491815E96
:100520009C4FFC018491882399F090E0880F991FDB
:10053000FC01E75EFC4FA591B491FC01ED5EFC4F20
:10054000859194918FB7F894EC91E22BEC938FBF47
:1005500008951F920F920FB60F9211242F933F937D
:100560004F935F936F937F938F939F93AF93BF93BB
:10057000EF93FF938091A3018F5F8093A3018091FC
:1005800062008111B2C08091610095B1E82FF0E066
:10059000E156FF4F90838230E1F1833009F450C07F
:1005A000811109C080919F00863978F1833A78F1F2
:1005B00082E08093600080919E008F5F863008F01B
:1005C00091C080939E00E0919E00F0E0E158FF4FC3
:1005D000808180936100806287B9369A8091620041
:1005E00091E0892780936200FF91EF91BF91AF91D5
:1005F0009F918F917F916F915F914F913F912F913B
:100600000F900FBE0F901F90189581E0D2CF80E021
:10061000D0CF8091A10090E0880F991F880F991F7B
:1006200020916000213011F4825D9109880F991F9B
:10063000880F991F01969093950080939400BBCFEB
:100640002091A20030E0220F331F220F331F409170
:100650006000220F331F220F331F413049F42F5AFD
:1006600034403695279530939D0020939C00A3CF6E
:10067000C9010196423049F5E091A000F0E045E063
:10068000F595E7954A95E1F790939D0080939C003E
:10069000ED59FF4F608170E001965BD190939B0014
:1006A00080939A00608570E0C901029752D19093BF
:1006B000990080939800608970E0C901089649D13B
:1006C000909397008093960076CF90939D008093AF
:1006D0009C0090939B0080939A0090939900809344
:1006E000980069CF10929E006ECF8091600081309B
:1006F00009F473CF8091610090E0FC01E156FF4F57
:100700002081283C90F427B385589F4FFC0130810D
:1007100081E090E0A0E0B0E004C0880F991FAA1F1C
:10072000BB1F3A95D2F7822B87BB27B3E0916100BC
:10073000F0E0E558FF4F308181E090E0A0E0B0E0CC
:10074000AC01BD0104C0440F551F661F771F3A95C9
:10075000D2F74095422347BB28B3E0916100F0E017
:10076000E558FF4F308104C0880F991FAA1FBB1F97
:100770003A95D2F78095822388BB2FCF1F920F9294
:100780000FB60F9211242F933F934F935F936F9364
:100790007F938F939F93EF93FF938091890089BDFF
:1007A00080918C0088BD20919100309192008091C1
:1007B000940090919500280F391F30939200209358
:1007C000910080918A0090918B0040919C00509103
:1007D0009D00840F951F90938B0080938A00409119
:1007E0008F005091900060919A0070919B00460F8D
:1007F000571F5093900040938F0040918D0050916F
:100800008E006091980070919900460F571F509389
:100810008E0040938D0040916000411128C0892FC7
:100820009927FC01ED55FF4F80816091A00070E099
:1008300090E08FD0FC01E20FF31F56E0F695E795AC
:100840005A95E1F7FF27ED55FF4F8081809389008E
:10085000FF91EF919F918F917F916F915F914F9158
:100860003F912F910F900FBE0F901F90189525E08C
:10087000969587952A95E1F7809388008091860068
:10088000909187002091960030919700820F931FDE
:100890009093870080938600DBCF17B88FE886B9E6
:1008A000E3E9F2E083EA90E023E231E0DC01449105
:1008B0004D9331962A173B07D1F72FEF2093230151
:1008C000E2E2F1E0A4E2B1E020812D9331978E17AE
:1008D0009F07D1F78FB7F894C59A8FBF80E01ADED3
:1008E00081E018DE87B5826087BD87EC90E00197D4
:1008F000F1F700C0000007B400FEFDCF87B58460AB
:1009000087BD87B5806887BDF89483EA8ABD81E09A
:1009100083BF10BE1FBC82E08CBD8FEF8EBD8DBD2E
:1009200080E489BF84E880BF789417B88FE886B9DF
:1009300080E287B9369A87EC90E00197F1F700C022
:1009400000008091A3018C3010F40CDDFACF0ADD99
:10095000FECF0024552704C0080E591F880F991F89
:10096000009729F076956795B8F37105B9F7802D52
:08097000952F0895F894FFCFC4
:100978000101010202020301020404030405020149
:1009880005060803080708070608100502040300FF
:0609980001000200030053
:00000001FF
